:020000040000FA
:100000008A28040000000000EA230000EA23000020
:10001000EA230000EA230000EA230000EA230000AC
:10002000EA230000EA230000EA230000EA2300009C
:10003000EA23000006240000EA230000EA2300006F
:10004000EA230000EA230000EA230000EA2300007C
:10005000EA230000DC250000EA230000EA23000078
:10006000EA230000EA230000EA230000EA2300005C
:10007000EA230000EA230000EA230000EA2300004C
:10008000EA230000EA230000EA230000EA2300003C
:10009000EA230000EA230000EA230000EA2300002C
:1000A000EA230000EA230000EA230000EA2300001C
:1000B000EA230000EA230000EA230000EA2300000C
:1000C000EA230000EA230000EA230000EA230000FC
:1000D000EA230000EA230000EA230000EA230000EC
:1000E000EA230000EA230000EA230000EA230000DC
:1000F000EA230000EA230000EA230000EA230000CC
:10010000EA230000EA230000EA230000EA230000BB
:10011000EA230000EA230000EA230000EA230000AB
:10012000EA230000EA230000EA230000EA2300009B
:10013000EA230000EA230000EA230000EA2300008B
:10014000EA230000EA230000EA230000EA2300007B
:10015000EA230000EA230000EA230000EA2300006B
:10016000EA230000EA230000EA230000EA2300005B
:10017000EA230000EA230000EA230000EA2300004B
:10018000EA230000EA230000EA230000EA2300003B
:10019000EA230000EA230000EA230000EA2300002B
:1001A000EA230000EA230000EA230000EA2300001B
:1001B000EA230000EA230000EA230000EA2300000B
:1001C000EA230000EA230000EA230000EA230000FB
:1001D000EA230000EA230000EA230000EA230000EB
:1001E000EA230000EA230000EA230000EA230000DB
:1001F000EA230000EA230000EA230000EA230000CB
:1002000082280000000000008344550050000000D8
:1002100000277800000006000A0000008444520015
:100220004F5000003E007800000006000A00000069
:1002300084535700414200000080FD00000006008A
:100240000A000000834E4900500000000E87E800BD
:10025000000006000A000000C4545500434B000093
:100260001E27780010079800000006000C00000010
:10027000C4535700415000009E1F7800000F7800C3
:100280004F007800000006000E000000C44F56002A
:1002900045520000002778001E0090000000060074
:1002A0000C000000C3524F0054000000801F780073
:1002B0001E0090003E0F78004F27780000000600D7
:1002C00010000000C4504900434B00000000E9004A
:1002D000000040006E007800000006000E000000E4
:1002E000C4504F004B4500000000E90000004000F2
:1002F0000E0040003E0878003E0078000000060036
:1003000012000000C4524F004C4C00000000E900F5
:100310000C003400811F7800821F78008E0040009E
:1003200081004000911F7800010178000000E90081
:1003300000800900C21078004F0F78004F0178004C
:10034000CF0078003E007800000006002600000084
:10035000C43F4400555000000000B00001003200CE
:1003600000277800000006000E000000823E5200C8
:10037000801F78003E007800000006000A000000A0
:1003800082523E00002778004F00780000000600EF
:100390000A00000082524000002778007FB89700D2
:1003A000000006000A0000008140000010007800F4
:1003B0000000060008000000C24340001040780022
:1003C0000000FB00000006000A000000C121000040
:1003D0003E0878003E007800000006000A00000099
:1003E000C24321001E4878003E0078003E0078009D
:1003F000000006000C000000812B00003E004000C1
:100400000000060008000000C22B2B00811F7800AE
:10041000BE0078003E0040001E8F4800CF007800EC
:100420000000060010000000864E450047415400C1
:10043000450000000000EA00000006000C0000007B
:10044000812D00003E0010000000060008000000A2
:10045000C22D2D00811F7800BE0078003E001000E4
:100460001E8F1800CF00780000000600100000006A
:1004700082322A004100DD00000006000800000072
:1004800082342A004200DD0000000600080000005F
:1004900082322F004180DE000000060008000000CC
:1004A00082342F004280DE000000060008000000B9
:1004B00082303C004F80DE00000006000800000093
:1004C000C2303D000000B000010032000080EF00AB
:1004D0000080EA00000006000E000000C2303E006E
:1004E0000000B000020032000080EA004F80DE0011
:1004F000000006000E000000C2553C003E00100047
:100500000000EF00F2FF3900000006000C000000C0
:10051000C13C00003E0010000000EF00ECFF350081
:10052000000006000C000000C13D00003E00680015
:100530000000EF00E6FF3200000006000C000000A3
:10054000C13E00003E0010000000EF00E0FF3C0054
:10055000000006000C000000C34E4F0054000000D5
:100560000000B000DAFF32000000EF0000000600DB
:100570000E000000C2552A00811F78003E00B8001E
:10058000CF007800000006000C000000C12A000027
:10059000811F78003E80B900CF007800000006007F
:1005A0000C000000C5552F004D4F4400821F7800FD
:1005B000811F7800000178001E00780011000900FA
:1005C0000280D800010F7800CF0078004F0178003A
:1005D000000006001A000000C6552A002F4D4F00EB
:1005E00044000000821F7800811F7800000178001D
:1005F0003E0078001E00B800110009004288D800B3
:10060000010F7800CF0078004F017800000006004D
:100610001E000000C52A2F004D4F4400821F7800A5
:10062000811F7800000178003E0078001E80B9002C
:10063000110009004208D800010F7800CF007800AF
:100640004F017800000006001C000000C42F4D0080
:100650004F440000821F7800811F7800000178005D
:100660001E007800110009000200D800010F780078
:10067000CF0078004F017800000006001A0000004B
:10068000C12F0000811F780080007800F1FF070073
:1006900001F0A300010039008100EA00801F78000A
:1006A0003E00780000F0A300010039000000EA00DD
:1006B0004100DD00810050004F007800CF0078003D
:1006C0000500390000F0A300020031000000E8003E
:1006D000000006000000E9000000060030000000F5
:1006E000C34D4F0044000000DAFF07003E007800D1
:1006F000000006000C000000C22A2F00811F7800B5
:1007000080007800C5FF0700E1FF37000000060009
:100710000E000000C453510052540000831F7800A3
:10072000821F7800811F78000027EB00010820005D
:100730001E8140000211B8000200E10001003900F2
:100740001E8F40008100D100F9FF39001E01E80032
:100750001E11B8000010E100010031001E0FE8007A
:10076000CF0078004F017800CF0178003E0078007C
:100770000000060032000000C34D41005800000098
:100780001E00E10002003C003E0078000000060070
:10079000620747000000060012000000C34D490038
:1007A0004E0000001E00E100F9FF35003E00780019
:1007B000000006000E000000C3414200530000008C
:1007C0000000B00001003B000000EA00000006004D
:1007D0000E00000083414E00440000003E00600017
:1007E000000006000A000000824F52003E00700028
:1007F000000006000800000083584F00520000006F
:100800003E006800000006000A000000C3415300DB
:10081000480000000000B0000800320004003B0067
:100820000080EA00008009001E8FD100030037001D
:100830000000E900008009001E0FD0003E00780093
:10084000000006001E000000C34C530048000000DA
:100850000000B000F9FF3200F5FF3B000080EA0025
:10086000008009001E0FD100F4FF370000000600D1
:1008700016000000C3524F004C0000000000B00002
:10088000EEFF320004003B000080EA000080090017
:100890001E0FD300E9FF37000000E90000800900C7
:1008A0001E0FD200E5FF3700000006001E0000000A
:1008B00083434F004D0000000080EA000000060066
:1008C0000A000000C32B430021000000811F7800B4
:1008D000BE00780010C840003E007800CF007800CD
:1008E0000000060012000000C32D4300210000009C
:1008F000811F7800BE00780010C810003E0078000C
:10090000CF0078000000060012000000C22B21007A
:10091000811F7800BE007800108840003E007800FB
:10092000CF0078000000060010000000C22D21005A
:10093000811F7800BE007800108810003E0078000B
:10094000CF0078000000060010000000C4464900F7
:100950004C4C0000821F7800811F78003E01780017
:10096000BE0078000201E90002800900805878008A
:100970003E007800CF0078004F01780000000600AC
:100980001C000000C5434D004F564500821F7800F3
:10099000811F78003E0178009E001100BE007800A3
:1009A000050039000000E90009003300008009005B
:1009B00031597800060037000201400081004000F4
:1009C0000000E90002003300008009004161780066
:1009D0003E007800CF0078004F017800000006004C
:1009E00030000000C44D4F0056450000821F7800C3
:1009F000811F78003E0178009E001100BE00780043
:100A0000050039000000E9000B00330000800900F8
:100A1000311978000800370002014000020140004F
:100A200081004000810040000000E9000200330026
:100A300000800900412178003E007800CF00780056
:100A40004F01780000000600340000008449440093
:100A50004C4500000140FE00000006000A000000B6
:100A600085534C00454550000040FE000000060044
:100A70000A000000C8535F0054414D00504F4E0023
:100A80000027780000002100000006000E00000092
:100A9000C6535F00574F5200440000000027780003
:100AA00000062100000006000E000000C8535F0091
:100AB000464F52004D41540000277800000A2100A3
:100AC000000006000E000000C549540052583100D5
:100AD0000027780000102100000006000C00000034
:100AE000C55445004C4543000027780040102100C4
:100AF000000006000C000000C6434E00544954009C
:100B0000500000000027780060102100000006005F
:100B10000E000000C3504100440000000027780090
:100B200020112100000006000C000000C33E490017
:100B30004E00000000277800401121000000060050
:100B40000C000000C94D45004D5F44004550540065
:100B50004800000000277800601121000000060016
:100B600010000000CB4D45004D5F5000524748003B
:100B70004552450000277800801121000000060042
:100B800010000000CA414400525F4300524541003A
:100B90005445000000277800C01121000000060025
:100BA00010000000C5535400415254000027780043
:100BB00000122100000006000C000000C554450092
:100BC0004D5053000027780040122100000006001D
:100BD0000C000000C5544100434845000027780040
:100BE00060122100000006000C000000C84D450006
:100BF0004D5F4800455245000027780080122100D3
:100C0000000006000E000000CA5354004F505F0061
:100C1000464F52005448000000277800A0122100DF
:100C20000000060010000000C4454F004C4E0000BC
:100C300000277800E0122100000006000C000000F0
:100C4000C3454F0046000000002778000013210034
:100C5000000006000C000000C442410053450000A3
:100C60000027780020132100000006000C0000007F
:100C7000C55354004154450000277800401321001B
:100C8000000006000C000000C5455200524F520003
:100C90000027780060132100000006000C0000000F
:100CA000C9545F005355530050454E0044000000A6
:100CB00000277800C013210000000600100000008B
:100CC000C8505200494F520049544500002778004F
:100CD000E0132100000006000E000000CA494E008B
:100CE000505554005F4649004C45000000277800ED
:100CF000001421000000060010000000C750520040
:100D0000475F50004E54000000277800401F21002C
:100D1000000006000E000000C54445005054480085
:100D200000277800E03F22000E0050004180DE00E6
:100D30000000060010000000C65244004550540058
:100D40004800000000277800402022000080570063
:100D50004180DE000000060012000000C750520073
:100D6000474845005245000082FF070000277800F1
:100D7000801F78003E0078002000B000100078004E
:100D8000002778004F00780010007800000006006F
:100D90001C000000C83E5000524748004552450024
:100DA00074FF070000277800801F78003E0078005D
:100DB00087FD0700002778004F0078002000B00072
:100DC00083FD0700000006001C000000C4454D0024
:100DD00049540000002778000027780030012000E7
:100DE000D2FD07002BFD070000277800100120002E
:100DF000CEFD07003E007000D9FD07000000B000E6
:100E00003E0078001E00320037FF07001000780017
:100E10000000B0003E0078000E003200002778008D
:100E200080BB200030FF070069FD07000027780025
:100E3000A0002000BDFD07000000B0003E007800CB
:100E40000300320000277800E00220000100370094
:100E500000000600002778000000B0003E00780087
:100E600007003200A1FF07002008B00053FD070073
:100E700094FD07000000B0003E007800F9FF32004A
:100E8000002778000000280090FF07000027780066
:100E9000801F78003E00780000277800100078005E
:100EA000801F78003E00780049FD07000027780089
:100EB0002022200010007800002778000020200069
:100EC0003E0060000000B0003E00780003003200E9
:100ED0000027780000002000050037000027780078
:100EE000402220003AFD070000277800F0FF2F0085
:100EF0000000B0003E007800ECFF320000277800D0
:100F00004F007800002778004F00780030FD070080
:100F100000000600A6000000C45052004740000038
:100F200079FF0700811F7800821F7800831F7800F7
:100F3000BE0078001000A7001600370002802F00C6
:100F4000028160001010E10012003A0010019000D0
:100F50001E10E1000F003A004000B000E37F2000C7
:100F60008380600000804000C108DE0000804000F7
:100F70000001EB000000A600B000780030417800CE
:100F80000000A600B0007800020F78000100780091
:100F900005003700420520001E0978001181BA00C3
:100FA000020F78001100BA00CF0178004F017800DD
:100FB000CF0078000000060052000000C45052002C
:100FC0004721000050FF0700811F7800821F780032
:100FD000831F7800BE00780002802F00028160002D
:100FE0001010E10003003A00100190001E10E10013
:100FF000060032001000A6002A00070002802F0021
:10100000029860001E107800130007004000B00036
:10101000E37F20008380600000804000C108DE0084
:101020000080400062074700BE0078003E01780063
:101030000000A60001187800025878000000A60001
:10104000011878003E007800CF0178004F01780049
:10105000CF00780000000600811F7800821F780012
:10106000831F7800841F7800B000780042052000BC
:1010700030097800F31F20001101BA003182BA0054
:1010800002187800045878001101BA003182BA00C1
:1010900004587800021878008301E900F6FF310057
:1010A00029003700811F7800821F7800831F780095
:1010B000841F780021042000020E2000911F780078
:1010C00091087100B0007800320024004239880095
:1010D00042052000300978008108BB00520520003D
:1010E00072398800A20A20007239880029E7A80016
:1010F0000000000000000000F31F20001200240088
:101100004239880030017800304278008208BB0004
:101110008498BB0030427800300178008208BB0020
:101120008498BB005205200072398800A20A200072
:101130007239880029E7AF00FEFF37008301E9001C
:10114000EEFF31004200F90041C020000080100095
:101150004F027800CF0178004F017800CF0078006F
:1011600000000600D6000000C4505200472C0000CA
:10117000FDFE070047FC070046FC0700002778003B
:101180000000200000277800200020009FFC0700BE
:1011900003FF07008BFF0700000006001C00000093
:1011A000CB7370005F7379006E637000726721000B
:1011B000D5FE07001000A600BAFF07001000A0002F
:1011C0003E0078000000060032000000C4484500E0
:1011D0005245000088FE070010007800000006005D
:1011E0000C000000C53E48004552450082FE070045
:1011F00077FC0700000006000C000000C2432C0032
:10120000F4FF0700002778001000B000F7FF070088
:1012100074FC07000000060010000000C12C000054
:10122000ECFF0700002778002000B000EFFF070068
:1012300067FC07000000060010000000CA73700081
:101240005F636F006D7069006C65000011FC070042
:1012500010FC070032FF0700801F78003E00780076
:10126000002778003E006800002778007FB89700CC
:1012700000277800F00320003E0060001000B0005E
:101280000027780030002000F2FC0700FAFB07007E
:1012900093FC07003E0010004100DD005BFC0700EE
:1012A000002778004F007800002778000004200015
:1012B0003E0060000000B0003E00780031003200C7
:1012C000A9FE070000277800000020000027780012
:1012D000200020004DFC07005EFC0700EDFB07002E
:1012E00000277800F0FF2F0090FC07000000B000FE
:1012F0003E0078000D003200801F78003E0078002C
:101300003E00780000277800700020000027780059
:101310004F0078004180DE000027780000002800A0
:101320003E00700092FF0700150037008EFE070098
:10133000002778000000200000277800200020000F
:1013400032FC070031FC0700801F78003E00780067
:101350000027780020002000002778004F00780048
:1013600083FF0700801F78003E0078000027780088
:1013700000002000002778004F0078007CFF070065
:1013800017003700C3FB0700C2FB0700E4FE07009D
:1013900077FF070000277800000020000027780072
:1013A0002000200019FC0700BAFB0700B9FB07006A
:1013B000DBFE070043FC0700AFFB070000277800B7
:1013C0006000200059FC07003E0060000000B000F3
:1013D0003E007800EBFF32003E0078003E007800CF
:1013E00000000600E60000004249460000277800A1
:1013F000000B200000277800000020005CFF0700A1
:10140000002778008007200000277800E0032000F4
:1014100057FF0700002778002003200000277800EE
:10142000F0FF2F0052FF07004FFE070000000600EC
:1014300026000000C77370005F73610075740000C0
:10144000801F78003E007800801F78003E00780002
:1014500090FB07008FFB07000027780000002000AA
:101460000027780020002000FAFB0700ACFE0700F0
:101470003E007800002778004F00780000277800B1
:101480004F00780000277800500020008FFB0700F5
:1014900000277800500020008CFB0700EDFB0700C0
:1014A000801F78003E00780000277800F0002000C0
:1014B000E7FC0700002778004F007800002778003D
:1014C000F0FF2F00E2FC07003E00400000277800FC
:1014D000400020008DFB070000277800400020001E
:1014E0008AFB070000277800000020000027780012
:1014F00020002000D7FB0700B2FE07000000060016
:101500008E00000044454C00534500000027780041
:101510007003200000277800F0FF2F0014FF070061
:1015200011FE0700C6FF07000FFE070000000600BF
:101530001800000044544800454E00000AFE070011
:10154000BFFF0700000006000C00000044434100FC
:101550005345000000277800000020000027780095
:10156000002778000000200000277800601B200082
:1015700036FF07000000060018000000424F46003A
:10158000002778000000200000277800A01C200021
:101590002EFF0700002778000000200000277800B9
:1015A0004029200029FF070090FF070000000600E7
:1015B0001C00000045454E00444F4600D3FF070085
:1015C000000006000A00000047454E004443410069
:1015D00053450000D2FD07004180DE005EFB07009E
:1015E0000000B0003E00780025003200002778009F
:1015F0003000200035FB0700002778003000200075
:1016000032FB07003E0070000000B0003E00780092
:1016100008003200801F78003E007800D2FD0700ED
:1016200087FF0700002778004F0078001000B10006
:10163000020037003E0078003E0078000027780066
:10164000A0FB07000000B0003E007800E7FF32007A
:101650003E00780000277800000020000027780076
:10166000001C2000F9FE0700002778000000200081
:1016700000277800E0102000F4FE07000200370089
:1016800000277800F0FF2F00000006006400000033
:101690004542450047494E00B3FD070000000600E3
:1016A0000A00000045554E0054494C004FFF07000A
:1016B000002778004000200014FB07000027780076
:1016C0004000200011FB07005DFF0700000006003E
:1016D0001800000045574800494C450043FF0700EB
:1016E000000006000A000000465245005045410037
:1016F0005400000085FF070000277800400020000C
:1017000002FB07000027780040002000FFFA0700D6
:101710004BFF0700000006001A00000042444F0083
:1017200000277800000020000027780080132000A8
:10173000C6FE07008CFD070000277800000020008F
:1017400000277800601B2000C0FE070000277800FB
:101750000000200000277800601B2000BBFE07006F
:101760000000060026000000452B4C004F4F5000A3
:10177000002778000000200000277800001C2000CF
:10178000B2FE070000277800000020000027780044
:10179000C01F2000ADFE07000027780000002000D9
:1017A00000277800001C2000A8FE07000027780012
:1017B000000020000027780060142000A3FE07002E
:1017C0000027780000002000002778006014200027
:1017D0009EFE070000277800000020000027780008
:1017E0008028200099FE07000027780000002000D4
:1017F00000277800C02A200094FE0700ABFF0700F6
:10180000002778000000200000277800E01020006A
:101810008EFE0700002778000000200000277800D7
:10182000E010200089FE07000000060064000000B0
:10183000C74C490054455200414C00000027780035
:1018400080072000002778000070220048FE070073
:1018500000277800801F78003E007800002778007D
:1018600040FF2F00FAFB07000002B00000277800BD
:101870004F0078000027780040002000F4FB0700AC
:101880003BFE07004AFE0700000006003000000093
:10189000444C4F004F5000000027780010002000FB
:1018A000E6FF0700B2FF070000000600100000007E
:1018B00081490000002778007FB8970000000600EB
:1018C0000A000000814A0000002778005FB89700F6
:1018D000000006000A000000814B0000002778008D
:1018E0003FB89700000006000A000000854C450044
:1018F00041564500002778004F0078004F007800DF
:10190000801F7800801F78003E00780000000600ED
:1019100014000000844558004954000000000600EF
:1019200008000000C243520000277800D0002000C9
:1019300028FD070000277800A000200025FD0700F3
:101940000000060012000000C44245004C4C00009C
:1019500000277800700020001EFD07000000060030
:101960000E000000C5535000414345000027780099
:101970000002200017FD0700000006000E00000016
:10198000C6535000414345005300000072FA07005F
:101990000000B0003E00780008003200F3FF0700AE
:1019A0001000B10000277800C6FA07000000B00060
:1019B0003E007800F9FF32003E007800000006008B
:1019C00022000000C4545900504500000027780050
:1019D000C3FA07000000B0003E0078002F0032007C
:1019E0001000B100801F78003E00780000277800CA
:1019F00072FA070000277800F00F20003E00600018
:101A000000277800AFFA070022FA070000277800C5
:101A100030002000C5FA07003E0070000000B00052
:101A20003E007800090032003E0078000027780070
:101A30004F0078003E00780000277800000020006A
:101A4000801F78003E0078000B00370000277800E8
:101A500000277800D0002000B4FA07000000B00092
:101A60003E007800030032003E007800AEFF070021
:101A700001003700D7FC07001000B00000277800F5
:101A80004F007800002778008EFA07000000B000B1
:101A90003E007800D2FF320069003700002778004E
:101AA0004F80DE000000B0003E007800640032008D
:101AB000801F78003E007800F6F90700F5F907006E
:101AC00017FD0700002778004F0078000000EA00AB
:101AD000002778000000B0003E00780014003200BB
:101AE000801F78003E0078000027780080FF2F00DC
:101AF00057FB07000027780000277800D00020005F
:101B00008AFA07000000B0003E00780003003200AF
:101B10003E00780084FF070001003700ADFC07009D
:101B2000002778004F0078001000B1000200370055
:101B3000D1F907003E00780000277800801F780068
:101B40003E0078000000B0003E0078001100320036
:101B50000027780000277800D000200073FA0700E3
:101B60000000B0003E007800030032003E00780024
:101B70006DFF07000100370096FC07000027780082
:101B80004F0078001000B100801F78003E00780000
:101B9000010037003E007800002778000000200098
:101BA000002778002000200018FA0700B9F9070084
:101BB000B8F90700DAFC0700002778004F0078002A
:101BC000002778000000B0003E00780014003200CA
:101BD000801F78003E0078000027780000277800FA
:101BE000F00F20003E0060000027780000277800FA
:101BF000D00020004DFA07000000B0003E00780041
:101C0000030032003E00780047FF07000100370064
:101C100070FC0700002778004F0078001000B1002A
:101C20000027780027FA07000000B0003E00780087
:101C3000A7FF32003E0078003E0078003E007800AA
:101C40003E0078003E0078000000060046010000DB
:101C5000C5434F00554E5400002778001000B000D7
:101C600085F90700D5F9070000277800F00F20005C
:101C70003E0060000000060016000000C92D540060
:101C8000524149004C494E004700000000277800AF
:101C900013FA070000277800300020008BF90700B6
:101CA000002778003000200088F907001000B100FC
:101CB0003E004000C1F90700002778000002200024
:101CC0001AFA07003E0060000000B0003E007800F5
:101CD000020032001000B100ECFF370000000600E7
:101CE00034000000C34249004E0000000027780085
:101CF00020002000DAFB0700B5F90700000006000D
:101D000010000000C54F430054414C0000277800EC
:101D100080002000D2FB0700ADF90700000006009C
:101D200010000000C744450043494D00414C0000ED
:101D300000277800A0002000C9FB0700A4F90700D5
:101D40000000060012000000C348450058000000D3
:101D50000027780000012000C1FB07009CF9070064
:101D60000000060010000000C7434F004E5645001B
:101D7000525400001000B00000277800000020003E
:101D800044F907008DF90700002778000027780044
:101D9000B0022000E5F907000000B0003E00780026
:101DA000070032003E007800801F78003E00780077
:101DB0001000B000002778004F0078000C003700BA
:101DC00000277800D0022000D8F907000000B000FA
:101DD0003E00780006003200801F78003E00780048
:101DE0001000B000002778004F0078001000B1000C
:101DF000801F78003E007800002778006FF9070008
:101E00000003B100002778004F80DE000000B00022
:101E10003E007800040032003E0078000027780081
:101E2000F0FF2F00350037000027780000277800EA
:101E300090002000C3F907000000B0003E007800C9
:101E4000060032007000B1000027780000277800FB
:101E5000A0002000AFF9070002003700002778003B
:101E6000000020000000B0003E00780004003200B6
:101E70003E00780000277800F0FF2F001F00370099
:101E80000027780076FB070010007800A1F9070012
:101E90000000B0003E00780015003200801F78007E
:101EA0003E007800801F78003E0078006CFB070041
:101EB00010007800B0F90700002778004F00780084
:101EC0001000B000002778004F007800EAF8070003
:101ED000801F78003E0078003E0040000027780018
:101EE0004F00780000277800000020000300370032
:101EF0003E00780000277800F0FF2F000000B000BF
:101F00003E007800BCFF3200002778004F007800C8
:101F10000000B0003E00780005003200801F78000D
:101F20003E0078000000EA00002778004F007800AB
:101F300000000600E8000000C23C230000277800F3
:101F400000002000DCFA070026F9070000277800CF
:101F5000801F78003E0078004F80DE000027780068
:101F60004F00780016FA0700000006001C00000071
:101F7000C4484F004C440000CFFA07000027780007
:101F80001000B000002778001000B0000027780093
:101F900030002000CDF8070008F90700002778007E
:101FA000F00F20003E00600000277800E0052000D0
:101FB000FCF9070075FA070000277800FFF8070012
:101FC00000277800F00F20003E0060001000B000F5
:101FD00000277800E0052000F2F90700ADF80700BF
:101FE00000F907001000B000FEF80700000006002E
:101FF00042000000C123000019FB07001000780018
:102000006AF907009CF807000003B0000027780079
:1020100000277800900320004AF907000027780085
:10202000700020003E0060003E004000D2FF07002C
:102030000000060022000000C2235300EEFF07004C
:102040000027780046F907000000B0003E00780045
:10205000FAFF32000000060012000000C4534900DD
:10206000474E00008BF807000000B0003E007800EB
:102070000300320000277800D0022000BEFF0700D6
:102080000000060016000000C2233E003E0078005B
:102090003E00780088FA0700EFFE07000000060007
:1020A0000E000000C12E0000A4FF070000277800EA
:1020B00000022000B0FF0700E0FF0700E9FF070073
:1020C000F2FF070041FE07000000060016000000B6
:1020D000C13F000010007800F3FF07000000060079
:1020E0000A000000C2552E000027780000002000E2
:1020F00092FF070000277800000220009EFF0700E3
:102100003E0078005CF80700CCFF0700DFFF070007
:102110002EFE0700000006001C000000C4574F0000
:1021200052440000801F78003E0078005BFA0700F0
:10213000002778000000200056F80700A9F80700E3
:102140000027780000002000B9FA0700A0F8070077
:102150000027780000002000BBFA07009CF8070069
:102160006EFA07001000780072FA0700100078007D
:102170003E00400000277800801F78003E00780075
:102180001000B000002778001000200069FA070056
:10219000DFF90700002778004F00780087F8070074
:1021A00000277800F00F20003E0060000027780034
:1021B000801F78003E007800002778003000200063
:1021C00042F80700002778007CF807003E00400036
:1021D0001000B00083F80700002778004F00780057
:1021E00000277800B7F807002AF8070000277800D2
:1021F00030002000CDF807003E0070000000B00065
:102200003E0078000A0032003E0078000027780087
:10221000F0FF2F000027780085FA07006CF8070010
:102220000027780088FA070069F807002E003700B9
:102230000027780000277800D0002000BBF80700B6
:102240000000B0003E007800070032003E00780039
:1022500000277800F0FF2F000027780074FA0700AD
:102260005BF807002000370000277800801F780007
:102270003E0078000027780090002000ABF80700AF
:10228000002778007FB89700002778000002200020
:10229000A6F807003E007000002778004F00780085
:1022A000002778007FB89700A0F807003E00700074
:1022B0000000B0003E0078000300320000277800E4
:1022C000F0FF2F00080037000027780010002000E2
:1022D0000027780030002000FCF707007BF907009A
:1022E00000277800000020000000B0003E007800C9
:1022F000A0FF32003E007800002778004F007800F1
:102300003E00780000000600F8000000C127000031
:10231000002778000002200082FF070000277800D5
:1023200026F807000000B0003E007800CE00320022
:10233000801F78003E0078001CFA07000027780014
:10234000801F78003E0078002000B0001000780068
:10235000002778004F0078001000780000277800F0
:102360007FB89700002778000027780013F807004F
:102370003E0040001000B000002778004000200020
:10238000D2F707000027780040002000CFF70700B1
:10239000C0F70700BFF70700E1FA07000027780041
:1023A000F0F32F003E006000002778004F00780017
:1023B000B8F7070000277800F00F20003E0060000B
:1023C000B4F70700FDF7070000277800F00F2000A2
:1023D0003E00600055F807000000B0003E007800A5
:1023E000350032001000B0000027780060002000A7
:1023F000B6F70700A7F7070052F807000000B00083
:102400003E00780029003200A2F70700002778007C
:1024100080FF2F000EF907009EF70700E7F707007F
:1024200042F807000000B0003E0078001C003200B7
:102430001000B0000027780060002000A3F707001C
:1024400094F707003FF807000000B0003E00780056
:102450001000320000277800300020009BF70700B2
:102460008CF70700D5F7070030F807000000B00030
:102470003E007800040032001000B0000027780011
:10248000F0FF2F0002003700002778000000200036
:102490000200370000277800F0FF2F00020037000D
:1024A0000027780000002000020037000027780095
:1024B000F0FF2F0002003700002778000000200006
:1024C000801F78003E007800801F78003E00780072
:1024D0003E0078003E007800002778004F0078002A
:1024E000002778004F0078000000B0003E00780020
:1024F0001F003200002778004000200073F707001B
:1025000064F707000FF807000000B0003E007800F5
:102510000F003200801F78003E007800002778000E
:10252000000020000027780020002000B7F70700F7
:1025300058F7070057F7070079FA070000277800D7
:102540004F007800002778000000200007003700C7
:102550003E0078003E0078003E0078003E007800A3
:102560003E00780000277800F0FF2F003A00370087
:102570003E0078003E0078003E007800801F780022
:102580003E007800801F78003E00780041F7070089
:1025900040F707000027780000002000002778009F
:1025A00020002000ABF707005DFA070039F70700AD
:1025B00038F707003E0070000000B0003E007800D1
:1025C00017003200A3F70700002778004F007800BB
:1025D000002778004F007800002778004000200096
:1025E0003AF70700002778004000200037F707007F
:1025F00028F7070027F7070049FA070000277800A7
:10260000F0F32F003E0060000027780060002000FB
:102610002EF7070000277800000020000E0037008A
:10262000002778004F007800002778004F007800DE
:102630003E0078003E0078003E0078003E007800C2
:102640003E007800002778003E00680000277800F0
:1026500000277800F0FF2F000000B0003E00780057
:1026600053FF320003003700002778003E00680067
:102670000027780000000600B8010000C4464900A9
:102680004E44000022FF070002F7070001F7070091
:102690003E0070000000B0003E00780015003200DF
:1026A000FCF60700FBF607001DFA0700801F780004
:1026B0003E007800002778003E0068000027780080
:1026C0004F00780000277800F00320003E006000F3
:1026D0001000B0000027780030002000DDF7070070
:1026E000E5F607007EF707003E0010004100DD0020
:1026F00046F707000000060040000000415B0000B4
:1027000000277800000020005BF9070030F7070081
:10271000000006000E000000C15D000000277800E8
:10272000F0FF2F0054F9070029F70700000006000A
:102730000E000000C13A00000027780000022000CF
:1027400078FE070088F907000027780000002000C5
:1027500000277800200020002CF7070013F907005D
:1027600000277800801F78003E0078002000B0002D
:1027700010007800002778007FB8970010007800DC
:1027800034F707007AFA070077F907000027780086
:102790007FB897000EF70700002778004F007800F9
:1027A0002000B0000AF707000027780003F70700B1
:1027B00000277800F00320003E0060001000B00009
:1027C000801F78003E007800002778002000B000CD
:1027D000FAF6070000277800F00F20003E006000A6
:1027E000ACF607001000B000F4F6070000277800F0
:1027F0008000200016F80700002778007FB89700B7
:102800001000B10000277800000C20003E0070008E
:102810003E00400056FA07003000B0000027780064
:102820004F0078003000B100002778002CF7070037
:102830000000B0003E00780016003200801F7800D3
:102840003E007800002778002000B000DBF607008B
:1028500000277800F00F20003E0060008DF6070092
:102860001000B000D5F60700002778008000200097
:10287000F7F70700002778003000200093F60700E4
:10288000CEF6070000277800F00F20003E00600021
:10289000DFFF37003E0078003E0078000027780018
:1028A000F0FF2F00F4F80700C9F607001CF9070035
:1028B000A8F80700C6F6070000000600C6000000E2
:1028C000413B0000002778006000200000277800CE
:1028D0000000200026FA070035FA070000277800DC
:1028E00000002000E4F80700B9F607000CF9070023
:1028F00098F80700100078003E0010000000B000BB
:102900003E0078000E0032000027780030002000E2
:10291000DFF80700AEF6070080F807001000780027
:10292000DBF807002000B000A9F6070081F80700D7
:1029300010007800D6F807004000B000A4F60700A9
:102940000000060044000000C87370005F7461005E
:1029500063686500002778004F0078000027780042
:102960004F007800002778003000200057F607005D
:1029700000277800801F78003E0078008000B000BB
:1029800093F60700002778004F007800A000B00001
:102990008FF60700000006006E000000C6544100DC
:1029A000434845003A00000063FF070009FA0700AA
:1029B000A2FB0700002778000000200018FA07009B
:1029C000002778000000200015FA07000027780093
:1029D0000000200012FA0700002778000000200005
:1029E0000FFA070000277800000020000CFA07000B
:1029F000002778000000200009FA0700002778006F
:102A00000000200000277800404A21000FFA07004C
:102A1000000006003E000000C9545F004558450014
:102A2000435554004500000000277800801F7800BF
:102A30003E007800A000B000100078000027780069
:102A40004F0078008000B00010007800801F7800F0
:102A50003E007800801F78003E00780000000600ED
:102A600026000000C8545F00414A4F0055544500FD
:102A70008FF8070000277800801F78003E0078005C
:102A80001000780000277800F0FF2F000027780062
:102A90007FB897004EF60700801F78003E00780050
:102AA0004EF8070000277800100078002AF607008B
:102AB0000000B0003E0078003500320000277800AA
:102AC0003000200001F60700F2F5070097F6070036
:102AD0000000B0003E007800070032003E007800A1
:102AE0003E0078003E0078003E0078000027780025
:102AF000F0FF2F0025003700002778001000780035
:102B00000027780050002000F0F507007BF6070052
:102B10000000B0003E00780014003200002778006A
:102B200030002000E9F507004000B00028F607005B
:102B3000801F78003E00780000277800002778008A
:102B40004F00780022F6070000277800F0FF2F00E2
:102B5000D0F507002000B0001DF607001CF60700A6
:102B600000277800F0FF2F0008003700801F780052
:102B70003E0078003E007800002778004F00780083
:102B80004000B0000027780000002000130037004C
:102B9000801F78003E00780000277800002778002A
:102BA0004F0078000AF6070000277800F0FF2F009A
:102BB000B8F507002000B00005F6070000277800F0
:102BC00000002000B3F507004000B00000F6070049
:102BD000FFF5070000277800F0FF2F000000B0008D
:102BE0003E007800AFFF3200002778004F007800E9
:102BF000002778004F007800F5F507000000060078
:102C0000D0000000C8545F004143540049564500BD
:102C1000801F78003E007800002778001000200018
:102C2000D7F607000027780000002200DDF6070035
:102C3000002778004F0078006000B000E4F507003E
:102C40000000060022000000C9545F0050455200F9
:102C5000494F440045000000801F78003E00780086
:102C60000027780010002000C5F607000027780034
:102C700000002200CBF60700002778000000EA00E1
:102C8000002778007FB897006000B000D0F50700FB
:102C90004180DE00CBF70700100078003E004000C6
:102CA00000277800F0FF27003E0060000027780032
:102CB0004F0078002000B000C5F5070000000600B6
:102CC0003E000000C8545F00524554004952450080
:102CD000A1F507000000B0003E0078003D00320082
:102CE000F3F7070000277800801F78003E00780087
:102CF0001000780000277800F0FF2F0000277800F0
:102D00007FB89700B2F50700801F78003E0078007A
:102D1000B2F707005FF507005EF5070010007800C6
:102D200002F607000000B0003E00780015003200F7
:102D3000801F78003E007800002778000000200007
:102D400054F507006000B000A1F5070000277800E7
:102D50004000B00010007800002778004F00780095
:102D60009BF50700002778000000200049F50700C8
:102D70004000B00096F5070000277800F0FF2F0014
:102D80000B0037001000780073F507000000B0005A
:102D90003E007800040032004000B00000277800B8
:102DA000000020000200370000277800F0FF2F000D
:102DB0000000B0003E007800D6FF32003E007800F0
:102DC000002778004F007800002778004F00780037
:102DD0007FF50700000006008C000000C57370003E
:102DE0005F2E6700002778004F00780000277800EA
:102DF0004F00780027F5070026F5070048F8070080
:102E000000277800F00F20003E006000801F78004F
:102E10003E0078003E0078001EF507001DF5070013
:102E20000027780000002000002778007FB8970076
:102E30001000B000002778003000200005F60700E1
:102E40000DF50700A6F507003E0010004100DD006B
:102E50006EF50700002778004F00780006F50700A0
:102E6000801F78003E00780003F50700801F78007F
:102E70003E0078000000EA00D4FA070000000600D7
:102E8000E0000000C5544C004953540053F70700BC
:102E90001000780030F507000000B0003E00780018
:102EA0007000320000277800A000B0001000780009
:102EB000F8F407008000B0001000780000277800C8
:102EC00000002000002778002000200061F50700A6
:102ED000F0F40700EFF4070011F807003E00780057
:102EE000002778008007200090F507000000B00060
:102EF0003E007800F1FF320000277800000020003B
:102F0000002778002000200052F50700E1F40700B8
:102F1000E0F4070002F80700801F78003E00780008
:102F20003E007800002778004F00780000277800E6
:102F300000277800000820003E0060000000B0007C
:102F40003E0078000900320000277800F0032000DE
:102F50003E0060000000EA009CFA070083FA0700C8
:102F600000277800F0FF2F000200370000277800CC
:102F70003E0068000000B0003E007800DEFF320036
:102F800037F7070010007800801F78003E007800B7
:102F900067FB070093FF07000B707200696F7200F8
:102FA00069746500203A200000277800100078003E
:102FB0004DFC07002000B000002778004000B00062
:102FC00010007800002778004F80DE000000B0007D
:102FD0003E0078000B00320082FF07000D70650094
:102FE00072696F0064697100756520003A2078008D
:102FF0000000EA002CFC07007AFF0700026D730056
:10300000110037003E00780000277800100078009B
:103010004F80DE000000B0003E0078000600320065
:1030200070FF070009494E004143540049564500CE
:1030300020652000040037006AFF070007414300B5
:103040005449560045204500002778004F0078007D
:1030500003F70700DEF4070033FA07002000B00092
:103060008BFF370000000600F400000047434F00CC
:103070004D5049004C450000A5FC070085F40700B1
:1030800084F407003E0070000000B0003E007800AD
:103090000900320078F40700E8F90700E7F90700B3
:1030A000002778000000200000277800E091200031
:1030B00066F80700100037003E0078003E007800F8
:1030C0000027780030002000F1F60700C0F4070068
:1030D00092F6070010007800EDF607002000B0001F
:1030E000BBF4070093F6070010007800E8F607002D
:1030F0004000B000B6F40700000006004A000000DF
:10310000495B43004F4D5000494C45005D000000B5
:103110007FFC07005FF407005EF407003E007000CC
:103120000000B0003E0078000200320047F80700BF
:10313000100037003E0078003E007800002778003D
:1031400030002000D2F60700A1F4070073F6070054
:1031500010007800CEF607002000B0009CF40700B5
:1031600074F6070010007800C9F607004000B000B0
:1031700097F40700000006003E000000C745580015
:103180004543550054450000801F78003E007800FC
:10319000801F78003E00780000000600120000004A
:1031A000C12200000027780040002000B2F607008E
:1031B000D7F50700ECF6070000277800F00F200095
:1031C0000027780000002000000006001800000022
:1031D000422E2200002778000000200000277800FF
:1031E000E06E210019F80700EEFF0700000006005E
:1031F00012000000012800000027780020002000B5
:103200009DF60700C2F50700000006000E00000052
:10321000C22E5300C2F607004FF407000000B000B2
:103220003E0078001C0032000027780000002000DB
:10323000801F78003E007800002778001000B00062
:10324000002778007FB897003E0010001FF40700A9
:1032500095FB0700002778004F0078001000B000B1
:1032600000277800801F78003E00780009F40700EE
:10327000A8F40700BAF407000000B0003E00780090
:10328000EDFF3200002778004F0078003E00780004
:103290003E00780006003700D2FE07000C5069009F
:1032A0006C6520007669640065202100202078008C
:1032B000000006005400000049494D004D454400FF
:1032C000494154004500000038F607000027780007
:1032D000801F78003E0078002000B00010007800C9
:1032E000002778004F00780010007800E9F307000D
:1032F000E8F307000AF7070000277800F0F72F002F
:103300003E0060000027780040002000FFF3070027
:103310000027780040002000FCF3070029F7070091
:1033200000000600380000004644490052454300B2
:10333000540000001DF6070000277800801F780069
:103340003E0078002000B0001000780000277800D0
:103350004F00780010007800CEF30700CDF307008F
:10336000EFF6070000277800F0FB2F003E0060001A
:103370000027780040002000E4F3070000277800D1
:1033800040002000E1F307000EF7070000000600F0
:1033900036000000C5414C004C4F54000027780017
:1033A0000000B0003E0078000500320000277800E1
:1033B000000020009AF707001000B100F7FF370067
:1033C0003E007800000006001C000000C44C4F00C6
:1033D000414400002EF60700100078000000B00005
:1033E0003E007800020032003E007800F501370010
:1033F00036F6070010007800801F78003E00780045
:10340000002778001000200030F60700F0F30700D6
:10341000C2F5070010007800801F78003E00780099
:10342000C4F5070010007800801F78003E00780087
:10343000FFF5070010007800801F78003E0078003C
:1034400001F6070010007800801F78003E00780029
:10345000B2F50700DEF30700002778000000200027
:10346000B4F50700DAF3070003F607001000780050
:10347000002778001AF407000000B0003E00780032
:10348000B600320000277800200020002DF407004D
:103490000000B0003E007800A10032000027780054
:1034A000200220001FFB0700EBF90700002778002F
:1034B0003000200085F3070000277800F00F20007F
:1034C0000EF4070073F3070005F407003E006000E8
:1034D0000000B0003E0078002C003200801F780011
:1034E0003E007800801F78003E00780062F30700FD
:1034F00099F307000000B0003E007800170032008A
:10350000002778000027780000102000FBF3070058
:103510000000B0003E00780008003200002778006C
:103520007FB89700A5F307000027780080002000EF
:10353000C7F407003E00400007003700002778006E
:103540007FB897009DF307004BF3070008F70700CB
:1035500000277800000020000300370000277800D3
:103560007FB8970095F3070043F307001000B00001
:10357000002778004F0078001000B0000027780086
:103580004F0078001000B100C8FF37003E007800FF
:103590008AF3070000277800002778002002200027
:1035A000E2F307000000B0003E0078002A0032007D
:1035B0003E007800801F78003E00780066F3070028
:1035C0000000B0003E0078000400320000277800C0
:1035D0000000200028F30700E5F607002DF30700A0
:1035E0002CF307004EF607000027780000F02F00AC
:1035F0003E006000002778004F0078003E00400049
:10360000002778004000200030F3070000277800F2
:10361000400020002DF307006AF6070096F507002A
:10362000100078000027780030002000BFF307006A
:103630000000B0003E007800020032003E0078003A
:103640003E00780000277800400020008AF507003F
:10365000B7F40700310037007BF507001000780051
:103660000000B0003E007800030032003E00780009
:1036700000277800D000200006F30700002778001C
:10368000F00F20009DF307000000B0003E0078001E
:1036900021003200801F78003E007800F6F207001B
:1036A0002DF307000000B0003E0078001500320046
:1036B0000027780000277800001020008FF3070013
:1036C0000000B0003E0078000700320000277800BC
:1036D0004F00780000277800800020005CF407008D
:1036E0003E00400006003700002778004F007800B9
:1036F000E1F207009EF60700002778000000200096
:1037000002003700002778004F007800DAF2070047
:103710001000B000010037003E0078000E003700B6
:1037200000277800000220007EFA070010007800D1
:1037300000277800109022007CF307000000B00002
:103740003E007800040032000027780020002000AE
:1037500049F5070076F40700EB0037003E007800DB
:10376000EBFA0700CBF20700CAF207003E00700038
:103770000000B0003E0078005F0032003EF5070018
:10378000100078000000B0003E00780024003200F5
:10379000C0F20700BFF20700E1F50700B6F207002C
:1037A0003E00780000277800000820003E006000FE
:1037B0000000B0003E00780002003200A3F60700CF
:1037C00016003700B3F20700B2F20700D4F5070085
:1037D000801F78003E007800002778003E006800D7
:1037E000002778004F00780000277800F0032000C1
:1037F0003E0060001000B00000277800300020007C
:1038000094F307009CF2070035F307003E00100018
:103810004100DD00FDF207005BFE070035003700C8
:103820009CF207009BF20700BDF5070092F207002B
:103830003E00780000277800000C20003E00600069
:10384000002778000004200038F307000000B000D3
:103850003E007800110032003E0078003E00780003
:10386000002778002000200009F50700D8F20700A3
:10387000AAF407001000780005F507002000B0004A
:10388000D3F20700ABF407001000780000F5070042
:103890004000B000CEF20700160037007DF20700AE
:1038A0007CF207009EF50700801F78003E0078003C
:1038B000002778003E006800002778004F0078005D
:1038C00000277800F00320003E0060001000B000E8
:1038D00000277800300020005EF3070066F2070042
:1038E000FFF207003E0010004100DD00C7F20700B4
:1038F00025FE0700840037003E00780067F40700CB
:1039000000277800ADF207000000B0003E0078000C
:103910007B0032005FF207005EF2070015F9070036
:1039200062F207003E00780060F207003E00780077
:1039300000277800A1F2070000277800100220007D
:10394000F4F207000000B0003E00780008003200EA
:103950003E007800C8F40700100078000000B000B6
:103960003E00780001003200B4F707006300370022
:103970000027780091F207000027780000277800E0
:10398000B0022000E9F207003BF2070000277800B0
:10399000D0022000E5F207003E0070003DF2070073
:1039A0001000B00085F20700002778001002200008
:1039B000D8F207003E0060000000B0003E00780032
:1039C0003E00320033F207000000B0003E007800F5
:1039D0003700320079F20700A7F4070010007800E2
:1039E0000000B0003E00780027003200801F780001
:1039F0003E00780000277800002778000040200073
:103A0000BEF207000000B0003E0078000E00320059
:103A100000277800400020008DF307000027780081
:103A20004F00780000277800D0022000BFF2070086
:103A300000277800100020003E006000000BB0005E
:103A40000DF207000E0037007CF707000027780012
:103A500000042000002778004F007800002778003D
:103A6000D0022000B1F207000027780000032000F8
:103A70003E0060003E00100000277800E0032000B8
:103A8000BBF507000900370000277800B0022000CE
:103A9000A6F207000000B0003E00780002003200ED
:103AA0003E004000010037003E00100002003700D9
:103AB0003E0078003E007800100037003E0078009D
:103AC0003E007800002778001000200070F4070006
:103AD0003FF2070011F40700100078006CF40700B3
:103AE0002000B0003AF2070012F40700100078003E
:103AF00067F407004000B00035F20700020037000D
:103B00003E0078003E0078004FF407001000780077
:103B10005FF40700100078003E0070000000B00065
:103B20003E00780050FE32007DF407004F80DE003A
:103B30000000B0003E0078000E0032000027780040
:103B40004000200052F4070021F20700F3F30700C1
:103B5000100078004EF407002000B0001CF20700AF
:103B6000F4F307001000780049F407004000B000AB
:103B700017F20700002778004F00780032F40700A2
:103B800013F20700002778004F00780028F40700A0
:103B90000FF20700002778004F007800E5F30700D8
:103BA0000BF20700002778004F007800DBF30700D6
:103BB00007F20700002778004F00780043F4070061
:103BC00003F207000000060000040000C643520094
:103BD00045415400450000007EF5070017F7070037
:103BE00061F40700EBF3070000277800801F7800DE
:103BF0003E007800F6F10700002778004F007800BB
:103C00002000B000F2F107000027780040002000FB
:103C100000277800F0FF2F0055F5070000277800F7
:103C20000000200000277800F007200050F5070072
:103C30005FF507000000060038000000C873700040
:103C40005F646F0065733E00D2F3070000277800C1
:103C5000801F78003E0078002000B000100078003F
:103C6000002778004F0078001000780000277800C7
:103C700000002000002778004F007800002778001F
:103C80004000200091F1070000277800400020004C
:103C90008EF1070000277800000020000027780040
:103CA00020002000D9F10700C6F4070000277800A3
:103CB00040002000002778004F007800002778009F
:103CC0004000200091F1070000277800400020000C
:103CD0008EF10700BBF4070035F5070000277800D8
:103CE00000002000E4F30700B9F10700000006001F
:103CF0009400000045444F0045533E0000277800E3
:103D00000000200000277800E0E121004FF50700C7
:103D10000000060012000000C85641005249410050
:103D2000424C450084FA0700ABFF07003CF5070052
:103D3000C5FF07000000060012000000C8434F0046
:103D40004E535400414E54007BFA0700BBF6070067
:103D50000027780060002000002778000000200085
:103D600003F5070012F50700002778000000200087
:103D7000C1F3070096F107000000060022000000D2
:103D8000C653540052494E00470000006AFA07002B
:103D900039F10700A9F60700A8F607000027780008
:103DA000600020000027780000002000F0F40700E9
:103DB000FFF407000027780000002000AEF30700A2
:103DC00083F107000000060026000000C5564C00E5
:103DD0004953540075F3070000277800801F7800CE
:103DE0003E0078002000B000100078000027780026
:103DF0004F0078001000780026F1070025F1070039
:103E000024F1070023F1070045F40700801F780024
:103E10003E0078003E007800002778004F007800D0
:103E200000277800F00320003E0060000000EA0058
:103E3000E6F60700CDF6070016F1070015F10700BA
:103E400000277800000020000027780020002000D4
:103E500080F1070032F407000EF107000DF10700B2
:103E60003E0070000000B0003E0078000400320008
:103E700078F10700002778000000200004003700D8
:103E80003E0078003E00780000277800F0FF2F0009
:103E90000000B0003E007800D7FF32003E007800FE
:103EA0003E0078000000060070000000C34B450093
:103EB000590000008DF30700002778001000B000C3
:103EC0003EF107000140FE00F2F007003BF1070061
:103ED000F0F007003E0010000000B0003E00780047
:103EE000F8FF3200EBF007003E0040002000B00079
:103EF00032F10700801F78003E0078001000B0000B
:103F0000002778002DF107001000B000002778008E
:103F1000F00720003E006000D7F0070031F10700F5
:103F2000002778004F0078000000060042000000E3
:103F3000C5494E004B4559006CF307000027780037
:103F40001EF10700002778000027780030002000CD
:103F5000DEF007001000B00022F107001000B100F1
:103F600000277800F00720003E0060003E0040007F
:103F70002000B00011F1070000000600280000003A
:103F8000C84B450059424F004152440057F30700C7
:103F90001000B000002778001000B10007F1070002
:103FA000BCF0070005F107003E0010000000B00063
:103FB0003E0078000600320000277800FFF007007E
:103FC0003E0040001000B000FCF007000200370087
:103FD000002778003E006800000006003000000066
:103FE000C6455800504543005400000000277800A3
:103FF000F00F20003E006000002778000000200045
:104000000027780030002000B0F00700F5F007002E
:10401000A0F007001000B0009EF007000027780015
:10402000000220004BF20700A2FF070000277800E3
:1040300000277800F001200042F1070095F007000A
:1040400000277800F007200032F107003E006000F2
:1040500090F00700002778009000200033F107005F
:104060003E007000002778004000200097F0070015
:10407000D2F00700002778004000200093F00700EE
:1040800024F107003E0060000000B0003E00780010
:1040900047003200002778000027780090002000B9
:1040A00022F107000000B0003E0078001800320046
:1040B0003E007800002778000002200000277800EA
:1040C0008000200000277800400020007FF00700DB
:1040D000BAF0070000277800801F78003E007800C3
:1040E00000277800700020003E0060003E001000B5
:1040F000002778003000200074F0070000277800C7
:104100004F0078003E001000A6F1070002003700C3
:104110000027780010002000801F78003E00780003
:1041200000277800801F78003E0078000027780084
:1041300028F30700002778003000200063F0070014
:104140009EF007001000B00000277800400020001B
:104150005EF00700A3F00700002778003000200081
:104160005AF007000027780094F007003E00400056
:104170009CF00700002778004F00780000277800A7
:104180004F0078001000B10000277800CDF0070044
:104190000000B0003E007800DFFF32003E007800F3
:1041A0003E00780000277800000020004F00370014
:1041B0000027780000277800F0072000DBF00700D8
:1041C00034F007000027780080002000D7F00700B7
:1041D0003E0070002FF0070000277800C00120008B
:1041E000D2F007003E007000002778004000200059
:1041F00036F0070071F00700B9F007003E006000DC
:104200000000B0003E007800140032003E0078004C
:1042100020F0070069F00700002778001000200058
:104220003E001000002778003000200027F0070033
:104230006CF007000027780080002000E5F20700FE
:10424000CAF507000027780080002000E1F207008F
:1042500000277800000020002400370000277800A5
:104260000027780030002000B0F0070009F00700B8
:1042700000277800D0002000ACF007003E0070005E
:1042800004F007008FF007003E0070000000B0004F
:104290003E0078000B00320000277800300020003C
:1042A0000AF007000027780044F007001000B00073
:1042B0003E0040004BF0070000277800F0FF2F0081
:1042C0000A00370000277800A000200097F00700C0
:1042D000A3F007000000B0003E00780001003200AB
:1042E0009BF5070000277800000020000000B000C8
:1042F0003E0078004CFF32003E0078003E0078001F
:104300000000060094010000C4515500495400000B
:104310000F202200002778000000200000277800EE
:1043200055F207002AF0070059F2070028F00700AD
:1043300051F207001000780007F007000000B000FD
:104340003E00780015003200002778004F80DE0024
:104350000000B0003E007800040032003E0078000B
:1043600000277800A00320000B003700002778000A
:104370002000200073F007000000B0003E0078002D
:1043800003003200002778002002200002003700DE
:104390000027780080022000020037000027780004
:1043A000E00320008BF20700B5F10700002778003A
:1043B000CDF10700100078000000B0003E0078004A
:1043C0000300320000277800F005200002003700CB
:1043D00000277800E004200004FF070052F50700E2
:1043E0000027780030002000AAEF0700002778009F
:1043F000F2EF07003E0040001000B000F9EF0700A8
:104400000027780000002000A2EF0700F5EF07006A
:104410001000B000B4F10700100078000000B000F8
:104420003E007800080032000027780030012000AC
:1044300068F20700E7FB0700002778001001200062
:1044400064F2070001003700E2FB070010F20700EA
:10445000100078000000B0003E007800A00032009C
:104460000E402200A0F10700100078000000B0000C
:104470003E00780009003200C4FE07000000B000D2
:104480003E007800020032008AFE07003E007800FD
:104490000027780000002000020037000027780085
:1044A000F0FF2F000000B0003E007800EDFF32006A
:1044B000F1F107001000780000277800F0FF2F00CE
:1044C0001AF007000000B0003E0078002000320023
:1044D000B6F1070000277800801F78003E007800C2
:1044E0002000B00010007800002778007FB8970007
:1044F0001000780067EF070066EF070065EF070020
:1045000064EF0700002778000000200000277800F3
:1045100020002000CFEF070081F20700CDEF070059
:10452000002778007FB89700A9EF070000277800E0
:104530004F0078002000B000A5EF070018F2070038
:104540000027780000002000CBF10700A0EF070053
:1045500024FA0700052A2A002A2A20004FF1070022
:10456000BDF5070019F5070000F50700C8F10700C1
:104570001000780000277800002778001000200045
:10458000EAEF07000000B0003E0078000A003200A9
:1045900014FA0700183A2000496E7300747275000F
:1045A000637469006F6E2000494E43004F4E4E0009
:1045B00055452000217478000027780000277800F6
:1045C00020002000D9EF07000000B0003E00780076
:1045D0000A00320003FA0700193A2000496E7300FE
:1045E00074727500637469006F6E2000494D4D0050
:1045F00045444900415445002021780000277800B7
:104600000027780030002000C8EF07000000B0004D
:104610003E0078000B003200F2F907001B3A200040
:1046200050524F00424C45004D45200050696C00EF
:10463000652064006520520045544F00555220000B
:10464000210D54000027780000277800400020004A
:10465000B6EF07000000B0003E0078000B0032000B
:10466000E0F907001D3A200050524F00424C45002F
:104670004D45200050696C00652064006573200082
:10468000444F4E004E45450053202100002778003E
:104690000027780040002000AAEF07000000B000CB
:1046A0003E00780008003200CEF907000C3A2000E6
:1046B0004552520045555200206E6F0020696C0033
:1046C00079F60700010037003E007800A0F40700EB
:1046D00095F4070000277800F0FF2F000F00370047
:1046E00065F107001000780076EF07000000B000C9
:1046F0003E0078000700320000277800F004200018
:10470000B4F1070000277800B0042000B1F10700E1
:1047100085F4070000277800000020000000B000AA
:104720003E00780002FF32000027780000002000E1
:104730000000B0003E007800F5FE320000000600E8
:104740001E020000C54142004F5254000E4022009C
:1047500097F207000027780000002000002778006B
:104760005AF107001AEF07000027780050F1070000
:1047700017EF070000277800E8F0070014EF0700A4
:10478000ECF0070012EF070067F4070095F9070047
:10479000262A2A002A2A2000494E54004552520057
:1047A00055505400494F4E00204C6F00676963001C
:1047B00069656C006C652000284142004F5254002E
:1047C0002920210058F4070061F40700D0FE0700FB
:1047D0000000060000277800600320000027780012
:1047E000801F78003E0078001000780000277800D5
:1047F0004F0078000027780010002000C1F007006B
:1048000043F00700F2EE07000040060000277800A2
:104810006003200000277800801F78003E007800A9
:1048200010007800002778004F00780000277800FB
:1048300010002000E3F0070035F0070000277800A3
:104840000080200000277800801F78003E0078005C
:10485000100078000027780070FF2F003E006000F5
:10486000002778004F007800D9EE070010F107000C
:104870001000780013EF07000000B0003E00780041
:104880008C00320098F00700100078000000B000A3
:104890003E0078002C00320093F0070000277800DB
:1048A000801F78003E007800100078001000B100F2
:1048B00000277800002778004F007800C4EE07003A
:1048C00000EF07000000B0003E0078001E0032003C
:1048D00006F1070000277800B8EE07001000B000CE
:1048E00000277800F00720003E00600069EE070016
:1048F0001000B000B1EE070066EE07000BEF0700F6
:104900000000B0003E007800030032003E00780056
:104910003E0078000C00370000277800D00020000F
:10492000002778003000200068EE0700002778009C
:10493000A2EE07003E0040002000B000A9EE0700F4
:104940004DEE0700A7EE0700E0F00700100078002A
:10495000A2F0070010007800002778000000B000E7
:104960003E007800510032004AEE070049EE070091
:1049700010007800E1EE07000000B0003E00780073
:10498000450032008FF007001000780041EE07006C
:104990002000B00010007800002778004F80DE0073
:1049A000801F78003E0078003E001000002778004D
:1049B000000024003E006000002778004F007800CF
:1049C0003E007000E6EE07000000B0003E007800F8
:1049D000170032000027780010007800BBF00700B5
:1049E0007BEE0700002778000000280029EE070072
:1049F0002000B000C6EF0700002778004280BF000B
:104A0000002778007FF89700004EB20042E0B70020
:104A10003E0078001FEE070003F8070042E0B700F1
:104A20003E0078001BEE0700A8F0070068EE0700C4
:104A300064F00700811F7800821F78001001780061
:104A40009E0078008180E8001100E0000B003B0030
:104A5000210090000000E0000800320002003B004E
:104A60001100100003003700000041000001EB00BE
:104A7000A200980000F0A100800878003E007800B5
:104A80004F017800CF0078002000900000277800C8
:104A90008CEE07000200370000277800F0FF2F009F
:104AA0000000B0003E007800AFFF32003E0078000A
:104AB0003E00780085F0070010007800002778009D
:104AC000200020008DEE07000000B0003E007800BE
:104AD0003700320050F0070000277800801F780070
:104AE0003E00780010007800002778004F00780022
:104AF0002000B00010007800E6ED0700E5ED0700AB
:104B00003E0070000000B0003E0078002600320039
:104B10000027780000002000002778003EF0070002
:104B200000277800801F78003E00780028EE0700FC
:104B3000002778004F0078002000B00024EE070026
:104B4000F6EF0700100078000000B0003E0078008B
:104B50001200320000277800F00720003E006000BD
:104B6000002778004F0078000027780000F82F0019
:104B70003E0060003E004000002778004F007800B3
:104B80003E007800BCED0700801F78003E007800F2
:104B9000801F78003E007800020037003E00780059
:104BA0003E007800020037003E0078003E007800AA
:104BB00007EE070000400600002778006003200091
:104BC00000277800801F78003E00780010007800F1
:104BD000002778004F00780000277800602220002E
:104BE000F6ED0700002778000080200000277800FD
:104BF000801F78003E0078001000780000277800C1
:104C0000F07F2F003E006000002778004F00780002
:104C1000EFED0700AEEF070000277800801F780057
:104C20003E0078002000B0001000780000277800D7
:104C30004F0078001000780096ED070095ED070012
:104C40003E0070000000B0003E007800020032001C
:104C50004DF90700460037003E0078003E0078001E
:104C6000002778001000B1000000B0003E0078007E
:104C70003200320000277800002778003001200041
:104C80002AEE070083ED07000027780010012000BE
:104C900026EE07003E0070000000B0003E007800E5
:104CA0000700320000277800300120001FEE0700C7
:104CB0000EF007002008B000CAED07001E00370004
:104CC0000AF0070000277800BCED07001000B000D4
:104CD00000277800F00720003E0060006DED07001F
:104CE0001000B000B5ED07006AED07000FEE0700F9
:104CF0000000B0003E007800040032003E00780062
:104D00003E0078003E0078000B00370067ED07009A
:104D100000277800300020006CED070000277800A5
:104D2000A6ED07003E0040002000B000ADED0700FA
:104D300051ED0700ABED07000D00370000277800AC
:104D40003E00680000277800203A2200B2EF0700FA
:104D500000277800801F78003E0078009CED070057
:104D6000002778004F0078002000B00098ED070081
:104D700097ED0700004006001C030000D1544900D5
:104D80004D455200315F550041525400315F49009A
:104D90004E495400002778000000200000277800CA
:104DA000407420008AED070000277800E00320000F
:104DB000002778006074200085ED07000027780048
:104DC000F0642E00002778002010200080ED0700FE
:104DD00000277800000028000027780040102000FD
:104DE0007BED070000277800F007200000277800FF
:104DF0008022200076ED07000027780000002000C8
:104E0000BAEF070072ED0700002778008000280045
:104E100000277800002220006DED070000277800B1
:104E200000402000002778002022200068ED0700C5
:104E30000027780080802000002778000082200072
:104E400063ED0700002778000000280000277800A5
:104E5000208C20005EED0700002778000000200075
:104E600028EF07005AED0700000006007A00000056
:104E7000C55445004D504F0052EF07001000780018
:104E80000140FE0003ED07004EEF07001000780020
:104E900000277800300020000CED07003E001000D5
:104EA00096ED07000000B0003E007800F4FF3200ED
:104EB0003E0078003E007800000006002800000058
:104EC000C5464F0052544800C6F70700CC0D4500B8
:104ED0006E747200657A200064616E0073206C004D
:104EE00065206D006F6E64006520640075204600CB
:104EF0004F525400480D0D00202020002020430078
:104F00006F70790072696700687420006A706200CF
:104F10002E666F00727468000D0D4D00696372009B
:104F20006F2046004F525400482050004943320041
:104F3000344550002064730050494300333345002A
:104F4000500D20005665720073696F006E203100AD
:104F50002E3232002020640075203100362F3100BF
:104F6000312F3200303134000D202000687474007D
:104F7000703A2F002F6A7000622E66006F72740004
:104F8000682E6600726565002E6672002F0D200087
:104F9000206A7000625F66006F727400684079007A
:104FA00061686F006F6772006F757000732E630029
:104FB0006F6D0D000D205100756520006C6520009F
:104FC000464F520054482000736F690074206100FE
:104FD0007665630020544F0049210D000D696E0075
:104FE0000000060094000000C6464F0052474500EE
:104FF00054000000C6F40700A6EC0700A5EC07006B
:105000003E0070000000B0003E0078001D0032003D
:10501000A0EC07009FEC07000027780000002000AC
:1050200000277800200020000AED070099EC070017
:1050300098EC07005AEF0700B9EF070005ED0700ED
:10504000DAEE070000277800801F78003E00780025
:10505000DFEC0700002778004F0078002000B00048
:10506000DBEC070000277800F00F20000027780015
:10507000F0FF2F003CEF0700D2EF07004CF00700D5
:10508000020037003E0078003E0078000000060075
:1050900056000000CE5445004C45430048415200A4
:1050A00047454D00454E540001EF070000277800AA
:1050B000801F78003E0078001000780000277800FC
:1050C000F0FF2F00002778007FB89700C0EC0700A2
:1050D000801F78003E0078000027780080BB200009
:1050E00081EE0700BAEC0700002778004F00780037
:1050F000002778004F007800B5EC0700000006009C
:1051000038000000C94445004D415200524147005B
:10511000450000004035220020A0B7000F202200EB
:105120000E40220056EE07000027780000202100E4
:10513000002778000000200006EE07000027780016
:1051400010002000F0EE0700A1EC07000027780017
:1051500080DF210025F007000EFF0700FCF20700AA
:1051600000277800000020000027780000102000B1
:105170006BEF070047EC070046EC070000277800BC
:105180000000200000277800200020009FEC07008E
:1051900040EC07003FEC070061EF0700801F78003C
:1051A0003E00780000277800F00F2000DFEC0700B9
:1051B000002778004F00780000277800F0FF2F00CC
:1051C000DAEC07003E0060000000B0003E0078000E
:1051D000EAFF32002FEC07002EEC0700F0EE07008C
:1051E0002CEC0700002778005000200037EC070067
:1051F000CEEC070027EC07000027780050002000C5
:1052000032EC0700C9EC07003E0060000000B0006F
:105210003E007800050032003E0078003E00780035
:1052200000277800F0FF2F006900370019EC070015
:1052300018EC070000277800000020000027780005
:105240002000200083EC070035EF070011EC070079
:105250000000B0003E0078000A0032003E007800F6
:105260003E0078000027780000002000002778002A
:105270002000200077EC07000027780000002000C5
:1052800053003700801F78003E007800801F7800B0
:105290003E007800FFEB0700FEEB070000277800D8
:1052A0004F007800002778004F00780069EC070075
:1052B000F8EB07004F80DE000000B0003E007800F1
:1052C0000C0032003E0078003E0078000027780095
:1052D0000000200000277800200020005DEC07007F
:1052E000002778000000200000277800F0FF2F0042
:1052F00034003700E7EB070000277800700020003B
:10530000F2EB070089EC0700E2EB070000277800CA
:1053100070002000EDEB070084EC07003E00600009
:105320000000B0003E0078000A0032003E00780025
:105330003E007800DDEB07003E007800DBEB070065
:105340003E00780000277800F0FF2F00002778004B
:105350001C003700CFEB0700CEEB070000277800DA
:1053600000002000002778002000200039EC070012
:10537000EBEE0700C7EB07000000B0003E0078002E
:105380000E0032003E0078003E0078003E007800BB
:105390003E007800002778000000200000277800F9
:1053A000200020002BEC07000027780000002000E0
:1053B00000277800F0FF2F00020037000027780058
:1053C000000020000000B0003E007800B7FF32006F
:1053D0000000B0003E00780081FF3200ADEB070016
:1053E000ACEB0700F1ED070000277800801F780084
:1053F0003E007800F6EB0700002778004F007800A9
:105400002000B000F2EB0700A2EB0700A1EB0700C1
:10541000C3EE0700801F78003E0078000027780068
:105420001004200041EC0700002778004F007800AE
:105430000027780050CC24003CEC07003E006000C0
:105440000000B0003E007800200032000027780005
:10545000000020000027780020002000EBEB070070
:105460008CEB07008BEB0700ADEE0700801F780088
:105470003E00780000277800500420002BEC070045
:10548000002778004F00780000277800E0342400DF
:1054900026EC07003E0060000000B0003E007800EF
:1054A0000700320000277800000020000027780065
:1054B00020002000D5EB070033F70700020037007B
:1054C0003E0078003E007800020037003E00780081
:1054D0003E00780016F207007BFE07001CF1070073
:1054E0008BFB070000000600FFFFFF00FFFFFF002F
:00000001FF
